:100E0700000102030405060708090A0B0C0D0E0F63
:080E1700410010004100110030
:1009B80090E600E054E74410F000000090E604746C
:1009C80080F00000007406F0000000E4F000000071
:1009D80090E6107420F000000090E611F00000008E
:1009E80090E61274A2F000000090E61374A0F000E4
:1009F800000090E61474E2F000000090E61574E040
:100A0800F000000090E6047480F00000007404F028
:100A1800000000E4F000000090E6497482F0000055
:100A280000F000000090E6187410F000000090E656
:100A38001A7408F090E6917480F0000000F000004D
:100A48000090E695F0000000F000000043AF01229E
:1005B30078007C007D017BFF7A0E79077E007F1037
:1005C30012050DC204E5AA30E2030206E9E5AA30EA
:1005D300E7030206E975310075320490F400E02464
:1005E300FE700302068024FA700302069C2407604F
:1005F300030206C590FC007401F090F401E090FC46
:1006030001F090F402E090FC02F0D2B690F401E025
:10061300701AA3E0701630B01374C0120D2DC2B659
:100623007F08120D33D2B67F08120D3330B04690D7
:10063300E694E0FE90E695E07C002400FFEC3ECFDC
:1006430024FCCF34FFFE7B017AF47904120AE450D0
:100653001C90FC0330B4117408F07FE87E03120D84
:10066300357403120D2D80667404F0806190FC03D1
:100673007402F0805990FC037401F0805190FC00E7
:100683007402F0E4A3F0A3F030B406A37410F08076
:100693003D90FC037420F080357531007532119064
:1006A300FC007408F07A007B007D017F50120D6B13
:1006B3007F50120BB57AFC7B017D107F50120D4FDA
:1006C300800C75310075320190FC0074AAF0E5319D
:1006D30090E69CF0000000E53290E69DF0000000FB
:0606E30090E6957480F022
:0106E90022EE
:0C0D2D0090E601F07F147E007D007C0049
:100D39008F368E358D348C33783374FF120595ECEC
:060D49004D4E4F70F32235
:0A0AE4008E338F348B358A36893744
:100AEE00E4F538F539C3E5399534E53895335033A7
:100AFE00AB35AA36A937853982853883120533FF7F
:100B0E00E4FEC2B2EF1392B7EFC313FFD2B20EBE22
:100B1E0008F0C2B220B002C3220539E53970C6050D
:040B2E003880C2D376
:010B320022A0
:02004100D322C8
:02004E00D322BB
:02005000D322B9
:080E200090E6BAE0F51DD322B3
:100DE30090E740E51DF0E490E68AF090E68B04F08E
:020DF300D32209
:080E280090E6BAE0F51CD322AC
:100DF50090E740E51CF0E490E68AF090E68B04F07D
:020E0500D322F6
:0207FC00D32206
:0207FE00D32204
:0208FB00D32206
:100CE00090E6B9E0242F600D04701990E604E0FF4F
:100CF000430780800890E604E0FF53077F00000070
:070D0000EFF08002D322C3D3
:010D070022C9
:100D8700C0E0C083C082D2015391EF90E65D740149
:080D9700F0D082D083D0E032DD
:100DB700C0E0C083C0825391EF90E65D7404F0D029
:060DC70082D083D0E0326F
:100DCD00C0E0C083C0825391EF90E65D7402F0D015
:060DDD0082D083D0E03259
:100BED00C0E0C083C08285100C85110D850D8285F6
:100BFD000C83A37402F085080E85090F850F82857D
:100C0D000E83A37407F05391EF90E65D7410F0D04E
:060C1D0082D083D0E0321A
:100D9F00C0E0C083C082D2035391EF90E65D740828
:080DAF00F0D082D083D0E032C5
:1008BE00C0E0C083C08290E680E030E72085080C5F
:1008CE0085090D850D82850C83A37402F085100EAB
:1008DE0085110F850F82850E83A37407F05391EF58
:0D08EE0090E65D7420F0D082D083D0E0321F
:01003200329B
:01004A003283
:01005200327B
:0108FD0032C8
:0108FE0032C7
:0108FF0032C6
:010E38003287
:010E39003286
:010E3A003285
:010E3B003284
:010E3C003283
:010E3D003282
:010E3E003281
:010E3F003280
:010E4000327F
:010E4100327E
:010E4200327D
:010E4300327C
:010E4400327B
:010E4500327A
:010E46003279
:010E47003278
:010E48003277
:010E49003276
:010E4A003275
:010E4B003274
:010E4C003273
:010E4D003272
:010E4E003271
:010E4F003270
:010E5000326F
:010E5100326E
:010E5200326D
:010E5300326C
:100B7900C0E0C083C08290E6D1E0900010F090E61A
:100B8900D0E4F000000090E6D17402F000000053B8
:100B990091BF00000090E66104F000000090E69922
:0C0BA90004F075BB06D082D083D0E0328F
:010E5400326B
:0A07F20000010202030304040505E0
:10028D00E4F52CF52BF52AF529C203C200C202C2F2
:10029D0001D2B675B5C4D2B61209B8120E307E08A9
:1002AD007F008E0A8F0B751208751312750808756D
:1002BD00091C75100875114A751408751578EE54DA
:1002CD00C07003020396752D00752E808E2F8F3012
:1002DD00C374BC9FFF74089ECF2402CF3400FEE48C
:1002ED008F288E27F526F525F524F523F522F52102
:1002FD00AF28AE27AD26AC25AB24AA23A922A82171
:10030D00C31205825031AE23AF24E5302FF582E5BF
:10031D002F3EF583E0FDE52E2FF582E52D3EF5838D
:10032D00EDF0EF2401F524E43EF523E43522F5222A
:10033D00E43521F52180B9852D0A852E0B74002415
:10034D0080FF740834FFFEC3E5139FF513E5129E7D
:10035D00F512C3E50D9FF50DE50C9EF50CC3E50FEC
:10036D009FF50FE50E9EF50EC3E5099FF509E5080E
:10037D009EF508C3E5119FF511E5109EF510C3E537
:10038D00159FF515E5149EF514D2E843D82090E697
:10039D0068E0440BF090E65CE0443DF0000000E4C2
:1003AD00F5A2000000D2AFD20412000390E680E067
:1003BD0054F7F0538EF8C20390E6C2E054FBF00000
:1003CD00000000000090E619E054FEF000000090DF
:1003DD00E61BE054FEF000000090E6187410F000EB
:1003ED00000090E61A740CF0000000000000000000
:1003FD000090E6017403F01205B3300105120056AA
:10040D00C2013003F212004150EDC203120D08205B
:10041D00001690E682E030E704E020E1EF90E682FE
:10042D00E030E604E020E0E4120C8912004E80C7B3
:0B00360090E50DE030E402C322D3226D
:1000560090E6B9E0700302011514700302019224C0
:10006600FE700302021524FB700302010F147003D5
:100076000201091470030200FD1470030201032437
:10008600056003020279120050400302028590E6E1
:10009600BBE024FE602A14603B24FD601114602A34
:1000A60024067050E50A90E6B3F0E50B803C12009A
:1000B60036503EE51290E6B3F0E513802D02027449
:1000C600E50C90E6B3F0E50D8020E50E90E6B3F082
:1000D600E50F801690E6BAE0FF120CB5AA06A9074E
:1000E600EA49600DEE90E6B3F0EF90E6B4F0020256
:1000F60085020274020274120DF5020285120E28A0
:10010600020285120E20020285120DE302028512FA
:1001160007FC400302028590E6B8E0247F601514D0
:10012600601924027063A200E43325E0FFA202E412
:10013600334F8041E490E740F0803F90E6BCE054C6
:100146007EFF7E00E0D394807C0040047D01800227
:100156007D00EC4EFEED4F24F2F58274073EF583EA
:10016600E493FF3395E0FEEF24A1FFEE34E68F82A1
:10017600F583E0540190E740F0E4A3F090E68AF0BE
:1001860090E68B7402F00202850202741207FE40AA
:100196000302028590E6B8E024FE6016240260039E
:1001A60002028590E6BAE0B40105C20002028502A9
:1001B600027490E6BAE0705590E6BCE0547EFF7E8D
:1001C60000E0D394807C0040047D0180027D00EC39
:1001D6004EFEED4F24F2F58274073EF583E493FF5D
:1001E6003395E0FEEF24A1FFEE34E68F82F583E03F
:1001F60054FEF090E6BCE05480131313541FFFE046
:10020600540F2F90E683F0E04420F08072805F1256
:1002160008FB506B90E6B8E024FE60192402704E8D
:1002260090E6BAE0B40104D200805490E6BAE064E5
:1002360002604C803990E6BCE0547EFF7E00E0D33D
:1002460094807C0040047D0180027D00EC4EFEED32
:100256004F24F2F58274073EF583E493FF3395E06D
:10026600FEEF24A1FFEE34E68F82F583800D90E643
:10027600A08008120CE0500790E6A0E04401F09040
:06028600E6A0E04480F058
:01028C00224F
:0300330002004682
:0400460053D8EF326A
:100C890090E682E030E004E020E60B90E682E03076
:100C9900E119E030E71590E680E04401F07F147E29
:0C0CA90000120B3390E680E054FEF022B5
:1000030030040990E680E0440AF0800790E680E03F
:100013004408F07FDC7E05120B3390E65D74FFF03D
:0F00230090E65FF05391EF90E680E054F7F02203
:080E3000E4F51BD2E9D2AF2268
:100BB500AD0790E678E020E6F9C2E990E678E044F2
:100BC50080F0ED25E090E679F090E678E030E0F908
:100BD50090E678E04440F090E678E020E6F990E68B
:080BE50078E030E1D6D2E922EC
:100C5700AC0790E678E020E6F9E51B702390E6788C
:100C6700E04480F0EC25E090E679F08D16AF03A91B
:100C7700077517018A188919E4F51A751B01D3221C
:020C8700C32286
:100C2300AC0790E678E020E6F9E51B702590E678BE
:100C3300E04480F0EC25E0440190E679F08D16AFB6
:100C430003A9077517018A188919E4F51A751B0397
:040C5300D322C322C3
:03004B000206EAC0
:1006EA00C0E0C083C082C085C084C086758600C051
:1006FA00D075D000C000C001C002C003C006C00748
:10070A0090E678E030E206751B060207D490E67898
:10071A00E020E10CE51B64026006751B070207D4A2
:10072A00E51B24FE605F14603624FE70030207C5D1
:10073A0024FC70030207D1240860030207D4AB1714
:10074A00AA18A919AF1A051A8F82758300120533E0
:10075A0090E679F0E51A65167070751B05806B9046
:10076A00E679E0AB17AA18A919AE1A8E827583002A
:10077A00120560751B02E5166401704E90E678E07A
:10078A004420F08045E51624FEB51A0790E678E085
:10079A004420F0E51614B51A0A90E678E04440F0D1
:1007AA00751B0090E679E0AB17AA18A919AE1A8E44
:1007BA0082758300120560051A800F90E678E0447E
:1007CA0040F0751B008003751B005391DFD007D0E2
:1007DA0006D003D002D001D000D0D0D086D084D0A9
:0807EA0085D082D083D0E032FB
:020CB500A9078D
:100CB700AE14AF158F828E83A3E064037017AD0166
:100CC70019ED7001228F828E83E07C002FFDEC3EB0
:080CD700FEAF0580DFE4FEFF23
:010CDF0022F2
:100D4F00120C23E51B24FA600E146006240770F3BF
:0C0D5F00D322E4F51BD322E4F51BD322C1
:100D6B00120C57E51B24FA600E146006240770F36F
:0C0D7B00D322E4F51BD322E4F51BD322A5
:100D080090E682E044C0F090E681F043870100005D
:040D180000000022B5
:100B33008E318F3290E600E054187012E5322401B2
:100B4300FFE43531C313F531EF13F532801590E629
:100B530000E05418FFBF100BE53225E0F532E53114
:100B630033F531E5321532AE31700215314E600581
:060B7300120D1C80EE22B1
:100D1C007400F58690FDA57C05A3E582458370F9EA
:010D2C0022A4
:03004300020900AF
:030053000209009F
:10090000020D8700020DCD00020DB700020D9F0001
:10091000020BED000208BE000200320002004A0095
:10092000020052000208FD000208FE000208FF005B
:10093000020E3800020E3900020E3A00020E3B0091
:10094000020E3C0002004A00020E3D00020E3E0074
:10095000020E3F00020E4000020E4100020E420055
:10096000020E430002004A0002004A0002004A0050
:10097000020E4400020E4500020E4600020E470021
:10098000020E4800020E4900020E4A00020E4B0001
:10099000020E4C00020E4D00020E4E00020E4F00E1
:1009A000020E5000020E5100020E5200020E5300C1
:0809B000020B7900020E540055
:100800001201000200000040E4E411220000010295
:1008100000010A06000200000040010009022E004B
:1008200001010080320904000004FF0000000705F8
:10083000020200020007050402000200070586020A
:100840000002000705880200020009022E000101D3
:100850000080320904000004FF00000007050202C6
:100860004000000705040240000007058602400022
:10087000000705880240000004030904180358001B
:100880006F00720063006F006D0020004C00740068
:1008900064002E0028035800500044002800420045
:1008A000610073006500640020006F006E0020008E
:0E08B000410058005500500050002900000083
:03000000020A5899
:0C0A5800787FE4F6D8FD758139020A9F12
:10043D00E709F608DFFA8046E709F208DFFA803EA1
:10044D0088828C83E709F0A3DFFA8032E309F6088E
:10045D00DFFA8078E309F208DFFA807088828C83F6
:10046D00E309F0A3DFFA806489828A83E0A3F608AA
:10047D00DFFA805889828A83E0A3F208DFFA804C84
:10048D0080D280FA80C680D4806980F2803380105B
:10049D0080A680EA809A80A880DA80E280CA8033C4
:1004AD0089828A83ECFAE493A3C8C582C8CCC5833C
:1004BD00CCF0A3C8C582C8CCC583CCDFE9DEE7800C
:1004CD000D89828A83E493A3F608DFF9ECFAA9F08B
:1004DD00EDFB2289828A83ECFAE0A3C8C582C8CCE1
:1004ED00C583CCF0A3C8C582C8CCC583CCDFEADEFA
:1004FD00E880DB89828A83E493A3F208DFF980CC5C
:10050D0088F0EF60010E4E60C388F0ED2402B40454
:10051D000050B9F582EB2402B4040050AF232345FB
:06052D00822390048D738F
:10053300BB010CE58229F582E5833AF583E022507D
:1005430006E92582F8E622BBFE06E92582F8E222C7
:0D055300E58229F582E5833AF583E49322E1
:10056000F8BB010DE58229F582E5833AF583E8F0D1
:10057000225006E92582C8F622BBFE05E92582C87D
:02058000F22265
:10058200EB9FF5F0EA9E42F0E99D42F0E89C45F0CF
:010592002246
:100593007401FF3395E0FEFDFC080808E6CF2FF653
:1005A30018E6CE3EF618E6CD3DF618E6CC3CF6222C
:100A640002028DE493A3F8E493A34003F68001F219
:100A740008DFF48029E493A3F85407240CC8C33393
:100A8400C4540F4420C8834004F456800146F6DF62
:100A9400E4800B0102040810204080900E17E47ECD
:100AA400019360BCA3FF543F30E509541FFEE49357
:100AB400A360010ECF54C025E060A840B8E493A31E
:100AC400FAE493A3F8E493A3C8C582C8CAC583CA49
:100AD400F0A3C8C582C8CAC583CADFE9DEE780BE01
:010E1F0000D2
:00000001FF
